:020000000828CE
:08000800A90A9C0A0B11090072
:1000100000308600831600308600C5308100043031
:10002000850000309A008312A0308B0010308500CC
:100030000C3084008001840A841E1A28041E1A28A9
:10004000FB212130A5239D002430A523A0002230D0
:10005000A523A700A2000230A523AD001E30A523D2
:10006000AF002330A5239B009B18AB149B181B15D6
:100070000430A4002B120510CB21C520BA2080200B
:10008000E12009223D289C01642005194A289C187A
:100090005C284428642064206420A8010519A80A6B
:1000A000642064200519A80A642064200519A80AA0
:1000B0008511023028020800203089001E088800BF
:1000C0009523051D612821281A1873288611010C13
:1000D0007F3903196F281E02031C061108009E08B1
:1000E000031D061508000611010C7F3903197C2831
:1000F0001E02031C861108009E08031D86150800B9
:100100001408900015089100160892001708930033
:1001100094019501960197011430840092209B2050
:10012000A520080008309800051994284320800D68
:10013000980B94280800840A05199C284320800DF8
:100140000519A0284320800D0800840A0430980077
:100150000519A8284320800C840A0519AD284320DE
:10016000800C98030319B6288403A828800E840302
:10017000800E080020300519283E99000519BA287C
:100180006420990BBE2885110800AB1CDE282108CD
:100190001E02031CDC280310210C1B1821082F074A
:1001A0008F0029080F02031808002F0D29020318D9
:1001B000DB2805100800A901051408009B1805108C
:1001C0000800851510081402031D022911081502E4
:1001D000031D022912081602031D02291308170223
:1001E000031D022910081D020319FC281B1F0229E8
:1001F00010082002031D02296420120813020319AB
:100200009129032908002B161708FE3E03192A29F5
:10021000FF3E03190613FF3E03198613FF3E031921
:100220003029FF3E03197B21FF3E03196021FD3E6B
:1002300003193529FF3E03190617FF3E03198617D8
:10024000FF3E03192D29FF3E03198621FF3E0319A6
:100250006E21A9291208073C54291208F83E542996
:100260001208073C03184829542908301602031CB9
:10027000542903190229FD3E03190617FF3E0319ED
:100280008617FE3E03198621FF3E03196E21A92918
:1002900003196021FF3E03197B21FE3E03198613DB
:1002A000FF3E03190613A929130801391A06031979
:1002B000A929130801399A00032201309200A929C3
:1002C0009B1E6C29AB1E0800A8002230A523A700A6
:1002D000A200AB1228080800851008009B1E79298F
:1002E000AB1A0800A8000130A700A200AB1628082E
:1002F0000800851408001B1D84299B1C8229AB1053
:100300002B1108002B110800051008001B1D8F2958
:100310009B1C8D29AB142B1108002B15080005140C
:10032000080064201208013A031DA6292B189C29F5
:10033000FF30A3000430A4002B184D222B18A9294C
:100340002B149A0901309A050322A9292B1CA929EB
:100350002B106420CB211208013A0319C829120876
:10036000AA002B19C0290310AA0D9B1FC4299108AC
:100370000319C429111CAA0A9118C429AA0AC4295C
:100380002B1EC4293030AA072A08A523A100080083
:10039000A1019E0108001B1AED291A18DE29061278
:1003A00086169E08031986129B1D86162B1A0800B6
:1003B0009118DC2906130800061708008612061695
:1003C0009E08031906129B1D06162B1A0800911889
:1003D000EB2986130800861708001A18F52906125B
:1003E00091188616911C861208008612911806161E
:1003F000911C061208002030A5239E00A100253084
:10040000A5239A000800253089001A088800952342
:1004100008002708013C031D102A21089E0008003F
:100420002B1221081E0203190800A20B08002D0838
:100430001E020318242AA1080319212A2D089E0050
:10044000242A9E01A20A080021081E02031C2A2A4F
:100450009E032B2A9E0A2708A2009C012630A52372
:100460001E08AE00880B352A392AAE0703189C0AED
:10047000322A043088009C0CAE0C9C13880B3B2A5B
:100480009C080318452A9C0CAE0C2730A5232E0887
:100490000802031C0030A2070800A30B0800512A21
:1004A0000800FF30A300A40B0800872AA500A50AB6
:1004B0000B30AB1BAB2BA50B5E2A0800861606166D
:1004C000AB2386120612AB235B2A0230A5002F3025
:1004D000592A74221208013A0319692A742212084F
:1004E000013A031D6E2A0800BA2080201008140269
:1004F000031D742A11081502031D742A120816021E
:10050000031D742A13081702031D742A08000930FA
:100510005622013056226922B123A8030319B72AB3
:10052000A8030319BF2AA8030319C82AA80303199B
:10053000042BA8030319182BA80303196A2BA8037B
:100540000319722BA8030319492BA80303195A2B6B
:10055000A8030319282BA80303193B2B0430A80276
:100560000319822B100803198E2B65228B2A562221
:10057000692221308900100888009523892A562293
:10058000692222308900B123280888009523892A0E
:1005900056226922B123280889000310890D10080A
:1005A0000319E92A10302802031CD82A6522C92A17
:1005B0002808562269221008B1230310A80DA81F8D
:1005C000E32A6522DA2A280888009523013056227A
:1005D000C92A0630A500A523A800A5032503A52345
:1005E000A8020310280C8807250889009523831684
:1005F0008818F82A8312A50A1E3025020318892AB2
:10060000A50AA50A2508EB2A56226922B12304303F
:100610002802031C0D2B6522052B2330A523E73070
:100620008805A80328188815A81808169523892A6C
:1006300056226922B12303302802031C212B652294
:10064000192B2330A5238812281C88169523892A64
:1006500056226922B12304302802031C332B213097
:100660002802031C352B6522292B263089002808F7
:1006700088009523892A56226922B123A808031DE0
:10068000432B65223C2B27308900280888009523BE
:10069000892A56226922B12305302802031C522BD5
:1006A00065224A2B2330A523F830880528088804C2
:1006B0009523892A56226922B12303302802031C7C
:1006C000632B65225B2B2330A5238813281C8817F6
:1006D0009523892A5622692224308900100888002F
:1006E0009523892A56226922B12303302802031C4C
:1006F0007B2B6522732B2330A5230813281C081796
:100700009523892A6922B12303302802031C8A2BEE
:100710006522822BAB13281CAB17892AFF30A3005C
:100720000430A40001305622212883168B130812AE
:100730008811081555308900AA30890088140811DD
:100740008818A02B83128B170800890083160814C1
:100750008312080808009C019C029C08031DAD2B15
:100760000800A801901FB72BA80A101FA80A901E06
:10077000BD2B0330A807101EA807901DC32B0930FE
:10078000A807101DA807901CC92B1B30A807101C18
:06079000A807280808007C
:02400E00FB3F76
:104200000000000012000000140015001600180045
:104210001A001C001E0020002200250028002B0090
:104220002E00320036003A003E00430048004E00A7
:1042300054005A00600067006E0075007C000000AA
:1042400000002A0003002000A900000010001E004A
:10425000000000000000000000000000000000005E
:104260000000000008000A000C000E001000120000
:10427000150018001B001E002100250029002D003C
:00000001FF
